:020000040000FA
:020000002A28AC
:08000800A100030E8312A20007
:100010008B1305108510772105191028851D2328BD
:100020000519A01405192010851920148519A01090
:100030000519182885191828220E8300A10E210EF3
:100040000B108B174A28220E8300A10E210E0B10D5
:100050008B1709008316FF2390008312191499143B
:10006000191583163C30850083128B1583160C30CE
:10007000960083120B108B17A001850105148514BF
:100080006F21051085105B21051485146F21051063
:1000900085105B21A0184F282018D9284A28851AD6
:1000A000DB28051E612805148514672105108510BD
:1000B0005B21051485146721051085105B21A001C3
:1000C0004A280514772105107F2185147721851092
:1000D0007F210514772105107F2185147721851054
:1000E0007F210514772105107B2185147721851048
:1000F0007B210514772105107B218514772185103C
:100100007B2105147721051077218514772185102F
:100110007721051477210510772185147721851023
:100120007721051477210510732185147721851017
:10013000732105147721051073218514772185100B
:1001400073210514772105106F21851477218510FF
:100150006F210514772105106B21851477218510F7
:100160006B210514772105106721851477218510EF
:1001700067210514772105106321851477218510E7
:1001800063210514772105105F21851477218510DF
:100190005F215B215B210514851467210510851003
:1001A0005B21051485145B215B2105108510A001DE
:1001B0004A28851A5128051EE5280514851467214B
:1001C000051085105B21A0014A2805147721051030
:1001D0005F218514772185105F2105147721051093
:1001E000632185147721851063210514772105107B
:1001F0006721851477218510672105147721051063
:100200006B218514772185106B210514772105104A
:100210006F218514772185106F2105147721051032
:10022000732185147721851073210514772105101A
:10023000732185147721851073210514772105100A
:1002400077218514772185107721051477210510F2
:1002500077218514772185107721051477210510E2
:100260007B218514772185107B21051477210510CA
:100270007B218514772185107B21051477210510BA
:100280007F218514772185107F21051477210510A2
:100290007F218514772185107F215B215B21051447
:1002A0008514672105108510A0014A285B215B2178
:1002B0005B215B210800FA30A50087210800C830C7
:1002C000A50087210800AF30A500872108009630DF
:1002D000A500872108007D30A50087210800643033
:1002E000A500872108004B30A50087210800323087
:1002F000A500872108001930A500872108000A30D1
:10030000A500872108000130A500872108006E3074
:10031000A600000000000000000000000000A60B86
:080320008929A50B87290800BB
:02400E00943FDD
:00000001FF
